:103E0000281121411222421424441848281121412A
:103E100012224214244418484881412182422284BB
:103E20004424882810208000532811214112224266
:103E3000142444184830353A3F00020103080009B1
:093E400001040605070204030554
:10200000754901E549D39548500D740A123FD078BF
:1020100049740126F650EC22C201E52CD394054008
:1020200003752C00743090F202F0743C90F002F0D2
:102030007548C8122000A201B35008E52C64636003
:102040000280028063E52C90314FF8282873752CAC
:102050000190F102E0540364016002D201804775EF
:102060002C0290F100E0541564116002D201803618
:0D207000752C0390F001E054FC640C60023C
:10207D00D2018025752C0490F200E05403640360B6
:10208D0002D2018014752C0590F201E05401640117
:09209D006002D2018003752C637E
:10314F0002204E02205F0220700220810220920294
:02315F0020A3AB
:1020A600808E22E52CC3940475F00284FE7F008E98
:1020B6004974FE0E0323DEFDF548E54890F000F076
:1020C600052CE5495401B4000C90F402E065486023
:0520D60002D201800CA4
:1020DB0090F101E064F065486002D20122C201E593
:1020EB002CD394154003752C00743090F202F075CC
:1020FB0048C8122000A201B35008E52C64636002AB
:10210B0080030221EEE52C903161F8282873752CA1
:10211B000190F000E4F090F402E064006002D20160
:10212B000221EB752C0290F101E064F06002D20108
:10213B000221EB74FF90F000F0752C0390F402E099
:04214B0064FF6002CB
:10214F00D2010221EB752C0490F101E0640F6002C3
:10215F00D2010221EB1220A90221EB1220A9807CCF
:10216F001220A980771220A980721220A9806D12E7
:10217F0020A980681220A980631220A9805E1220F6
:10218F00A980591220A980541220A9804F1220A98A
:10219F00804A1220A980451220A980401220A980D0
:1021AF003B1220A98036752C15754A00E54AD39449
:0321BF00FF5024AA
:0121C200E537
:1021C3004A90F000F090F402E0654A6002D2019078
:1021D300F101E064F0654A6002D201784A74012695
:0821E300F650D58003752C6352
:1031610002211902212E02213E0221540221640270
:10317100216A02216F02217402217902217E02213A
:103181008302218802218D02219202219702219C32
:103191000221A10221A60221AB0221B00221B50226
:0231A10021E823
:1021EB0002210022754900754800AF48AE497D01B8
:1021FB007CFFECC39EED9F4063C20274002EF58200
:10220B0074403FF5837400F0AF48AE4974002EF56F
:10221B008274423FF5837400F0A202B3500280F93E
:10222B0090F001E05401AF48AE49FD74002EF582E9
:10223B0074403FF583EDF090F001E05402AF48AEEF
:10224B0049FD74002EF58274423FF583EDF0784919
:0A225B00740126F6500418E436F66C
:09226500508E22754C00754B00EF
:10226E007550FF754F00E548B40008904000E0F54A
:10227E004A8006904200E0F54A754E00754D00C248
:10228E0001AF4DAE4E7D027C00EE6C7004EF6D60C2
:10229E0005A201B34003022351E548B4000F7400B8
:1022AE002EF58274403FF583E0F5498011AF4DAEB7
:1022BE004E74002EF58274423FF583E0F549E549F0
:1022CE00B54A07784B123FF08071E54A6400602FE3
:1022DE00AF4BAE4C7414BF00039E5004D201801D50
:1022EE00AF4BAE4C740ABF0010D39E400CAD4FAC3A
:1022FE005074006C4D700280028002D201802DAFAE
:10230E004BAE4C7411BF00039E5004D201801DAF22
:10231E004BAE4C7406BF0010D39E400CAD4FAC506C
:0C232E0074006C4D700280028002D2012D
:10233A00755000754F00754C00754B0085494A78F9
:10234A004D123FF002228FAF4FAE5074006E4F60B5
:10235A0002D20122C201E52CD3940C4003752C0051
:10236A00E52CC394085006743090F202F0748B90F6
:10237A00F403F07548C8122000A201B35008E52CF6
:10238A006463600280030226B0E52C9031A3F8282A
:10239A002873752C01743C90F002F090F4007401DB
:0A23AA00F07548321220001221EFF6
:0123B40075B3
:1023B50053FF755200755100AF51AE527D017CFF40
:1023C500ECC39EED9F401F74002EF58274403FF5CF
:1023D50083E0FBEB5553F5537852740126F6500410
:1023E50018E436F650D2E553B40002D2010226AD08
:1023F500752C02743C90F002F0740290F400F075B4
:1024050048321220001221EF7553FF7552007551A5
:1024150000AF51AE527D017CFFECC39EED9F401F86
:1024250074002EF58274423FF583E0FBEB5553F5BE
:10243500537852740126F6500418E436F650D2E566
:1024450053B40002D2010226AD752C03743C90F002
:1024550002F0740290F400F0754832122000122147
:01246500EF87
:012466007500
:1024670048001222680226AD752C04747C90F00295
:10247700F0740290F400F07548321220001221EF38
:102487007553FF755200755100AF51AE527D017CF7
:10249700FFECC39EED9F401F74002EF58274403FF2
:1024A700F583E0FBEB5553F5537852740126F6504C
:1024B7000418E436F650D2E553B40002D2010226DE
:1024C700AD752C05743C90F002F090F4007401F0A7
:1024D7007548321220001221EF7548011222680256
:1024E70026AD752C0674BC90F002F0740290F400CF
:0124F700F0F4
:0124F800756E
:1024F90048321220001221EF7553FF7552007551B1
:1025090000AF51AE527D017CFFECC39EED9F401F91
:1025190074002EF58274423FF583E0FBEB5553F5C9
:10252900537852740126F6500418E436F650D2E571
:1025390053B40002D2010226AD752C07740390F43E
:1025490000F0743C90F002F07548C812200090F039
:1025590001E0540364036002D2010226AD752C0820
:1025690090F4007401F0743090F202F0747C90F0F1
:1025790002F07548C812200090F401E05403640386
:072589006002D2010226AD41
:0125900075D5
:102591002C0990F400E4F0742090F202F0747C9025
:1025A100F002F07548FF12200090F4007401F075FC
:1025B10048FF12200090F401E0540364016002D24C
:1025C100010226AD752C0A90F400E4F0743090F20B
:1025D10002F0754832122000743890F202F075480A
:1025E10032122000742890F202F0747C90F002F014
:1025F1007548FF12200090F4007401F07548FF1235
:10260100200090F401E0540364026002D20102262A
:01261100AD1B
:10261200752C0B90F400E4F0743890F202F07548D7
:1026220032122000743090F202F07548321220000B
:10263200742090F202F074BC90F002F07548FF1220
:0E2642002000740290F400F07548FF12200092
:1026500090F401E0540364016002D201804F752CB4
:102660000C90F400E4F0743090F202F075483212ED
:102670002000743890F202F075483212200074285D
:1026800090F202F074BC90F002F07548FF12200046
:06269000740290F400F05A
:102696007548FF12200090F401E0540364026002C2
:0726A600D2018003752C63D3
:1031A30002239C0223F502244E02246F0224C80248
:1031B30024E90225420225660225900225C502263E
:0731C3001202265E0226AA9B
:1026AD0002238322754D01A201B35009E54DC39458
:1026BD000A50028002805DE54D903E00123FE0E43D
:1026CD009390F302F090F002E0440190F002F07567
:1026DD004832122000E54AB4001390F000E0C454D3
:1026ED000FF54B90F001E05410F54C801090F00078
:1026FD00E0540FF54B90F001E05420F54CE54CB44F
:10270D000002800AE54B654D600280028002D20115
:04271D00054D809353
:10272100A201B3500A90F002E054FE90F002F022B0
:10273100741190F302F0754850122000E54AB4007C
:102741000D90F001E05440B40002D201800B90F0F2
:1027510001E05480B40002D20190F302E4F0754824
:0427610050122000F2
:10276500E54AB4000E90F001E0544064006002D2E6
:0F27750001800C90F001E0548064006002D201FA
:1027840022C201E52CD394054003752C0074929069
:10279400F003F0748B90F403F0743090F202F0754F
:1027A40048C8122000A201B35008E52C64636002FB
:1027B4008003022870E52C9031CAF8282873752C00
:1027C40001743C90F002F07548C812200090F001AA
:1027D400E054F064006002D20102286D752C02906E
:1027E400F4007401F090F300E4F0747C90F002F0D3
:0E27F4007548C8122000754A001226B1806B8D
:10280200752C0390F4007401F090F300E4F0747CF2
:1028120090F002F07548C8122000754A0012273164
:102822008049752C04740290F400F0741090F30047
:10283200F074BC90F002F07548C8122000754A018D
:102842001226B18026752C05740290F400F07410E3
:1028520090F300F074BC90F002F07548C8122000AA
:0B286200754A011227318003752C63BA
:1031CA000227C20227E00228020228240228470214
:0231DA00286A61
:03286D000227A996
:022870002275CF
:102872004B01A201B35009E54BC3940A50028002F6
:10288200805590F002E054DF90F002F0E54B903E6C
:1028920018123FE0E49390F000F0754850122000C7
:1028A20090F301E05410B40002D20190F301E0541D
:1028B2000F654B6002D20190F002E0442090F002DA
:1028C200F075485012200090F301E054106400604B
:1028D20002D201054B809B22C201E52CD394044015
:1028E20003752C00743090F202F0748B90F403F0B4
:1028F2007548C8122000A201B35008E52C64636039
:102902000280030229ABE52C9031DCF8282873758C
:102912002C01747C90F002F090F000E4F090F3004F
:0E292200E4F090F4007401F0754832122000C9
:1029300090F301E0540864006002D201806A752CB3
:1029400002745C90F002F090F300E4F090F40074F4
:1029500001F0754A00122871804E752C0374BE90E8
:10296000F002F090F000E4F090F3007401F07402D3
:0A29700090F400F0754832122000C8
:10297A0090F301E0540864006002D2018020752CB3
:10298A0004749E90F002F090F3007401F0740290C7
:0E299A00F400F0754A011228718003752C6359
:0F31DC0002291102293E02295A0229880229A537
:1029A8000228F822E54B903E24123FE0E49390F091
:1029B80000F0E54AB4000C90F002E054F790F00201
:0929C800F0800A90F002E054FBDB
:1029D10090F002F07401123FD090F002E0440C90AC
:0F29E100F002F075480112200090F000E4F0229F
:1029F000E54AB40008754EF7754F088006754EFB22
:102A0000754F04E54B90F000F090F002E0554E90C9
:102A1000F002F07401123FD090F002E0454F90F0C8
:102A200002F0754801122000E54C90F000F090F0A3
:102A300002E0554E90F002F07401123FD090F00287
:102A4000E0454F90F002F0754801122000E54D90EE
:102A5000F000F090F002E0554E90F002F074011298
:102A60003FD090F002E0454F90F002F0754801121F
:082A7000200090F000E4F022C8
:102A7800754A01E54AD395495045E548254AF54B3D
:102A8800E54BD394094007E54BC39409F54BE54B57
:102A9800903E29123FE0E49390F302F0752950E547
:102AA800296400600280F890F302E4F0752950E58B
:102AB800296400600280F8784A740126F650B4222E
:102AC800754A01A201B3500AE54904D3954A400268
:102AD8008003022B5E752978754C00E52964006037
:102AE80009E54C5410B400028002800890F301E01C
:0B2AF800F54C80E7E529B40004D20192
:102B03008034AF3DAE3E74002EF58274403FF583B2
:102B1300E54CF0783D123FF0E548254AF54BE54B8F
:102B2300D394094007E54BC39409F54BE54C540F87
:102B3300654B6002D201752978E5296400600C9029
:102B4300F301E05410640060028002800280EAE531
:102B530029B40002D201054A022ACB2290F002E0F6
:102B630054EF90F002F07401123FD090F002E04471
:0C2B73001090F002F075480A12200022B9
:012B7F00C293
:102B800001E52CD394074003752C00743090F202B9
:102B9000F0748B90F403F07548C8122000A201B3C2
:102BA0005008E52C646360028003022F38E52C9006
:102BB00031EBF8282873752C0190F000E4F0743C98
:102BC00090F002F0122B5F90F001E0540C640C6066
:102BD00002D201022F35752C02754A00754B001286
:102BE00029AC90F001E0540864006002D201743C0A
:102BF00090F002F0122B5F022F35752C03746C904D
:032C0000F002F0EF
:102C030090F4007401F0754832122000747C90F047
:102C130002F0743090F300F090F302E4F075480A88
:102C2300122000754A00754B021229AC754A0075D3
:102C33004B041229AC754A00754B001229AC740081
:102C4300F548754901122A78122B5F754A00754BB6
:102C5300041229AC754A00754B001229AC7400F5B7
:102C6300487401F549122AC8122B5F022F35752CBF
:102C730004746C90F002F090F4007401F075483223
:102C8300122000747C90F002F0743090F300F09006
:0A2C9300F302E4F075480A12200075
:012C9D0075C1
:102C9E005000E550D394035051754A00754B021203
:102CAE0029AC754A00754B041229AC7400F54AE53F
:102CBE0050903E35123FE0E493F54B7400F54C74A2
:102CCE0000F54D1229F0754A00754B001229ACE53E
:102CDE0050F548754906122A78754A00754B01124F
:102CEE0029AC7850740126F650A8755001E550D3E2
:102CFE009402500E7548FA1220007850740126F690
:102D0E0050EB755000753E00753D00122B5FA20111
:102D1E00B35009E550C3940450028002804B7548AD
:102D2E00FA122000754A00754B041229AC7400F596
:102D3E004AE550903E35123FE0E493F54B7400F5B2
:102D4E004C7400F54D1229F0754A00754B0012298E
:102D5E00ACE550F5487406F549122AC8754A007557
:0C2D6E004B011229AC055080A5122B5F10
:102D7A00022F357548FA122000752C05743C90F024
:102D8A0002F0754832122000122B5F754A01754B0A
:102D9A00001229AC90F001E0540464006002D201F0
:102DAA00122B5F022F35752C0674AC90F002F0746A
:102DBA000290F400F075483212200074BC90F002C0
:102DCA00F0743190F300F090F302E4F075480A12BF
:102DDA002000754A01754B021229AC754A01754BE0
:102DEA00041229AC754A01754B001229AC7400F51E
:0A2DFA0048754901122A78122B5F78
:102E0400754A01754B041229AC754A01754B0012C1
:102E140029AC7400F5487401F549122AC8122B5FD5
:102E2400022F35752C0774AC90F002F0740290F404
:102E340000F075483212200074BC90F002F0743136
:102E440090F300F090F302E4F075480A1220007544
:102E54005000E550D394035051754A01754B02124A
:102E640029AC754A01754B041229AC7401F54AE585
:102E740050903E35123FE0E493F54B7400F54C74EA
:102E840000F54D1229F0754A01754B001229ACE585
:102E940050F548754906122A78754A01754B011296
:102EA40029AC7850740126F650A8755001E550D32A
:102EB4009402500E7548FA1220007850740126F6D8
:022EC40050EBD1
:102EC600755000753E00753D00122B5FA201B35090
:102ED60009E550C3940450028002804B7548FA12EB
:102EE6002000754A01754B041229AC7401F54AE5B8
:102EF60050903E35123FE0E493F54B7400F54C7468
:102F060000F54D1229F0754A01754B001229ACE502
:102F160050F5487406F549122AC8754A01754B01E1
:0F2F26001229AC055080A5122B5F8003752C6318
:1031EB00022BB6022BD6022BFA022C71022D7D027A
:0831FB002DB0022E27022F3235
:102F3500022B9D22C201E52CD394034003752C007E
:0C2F4500743090F202F07548C8122000B1
:102F5100A201B35008E52C64636002800302314E84
:102F6100E52C903203F8282873752C01743C90F0FD
:102F710002F0754A00A200B350547529FAE529649C
:102F810000603F7480454A90F000F07548021220BD
:102F910000E54A04444090F000F075480212200018
:102FA100E54A2402442090F000F075480212200006
:102FB100E54A2403441090F000F075480212200005
:102FC10080BB054AE54AB40B03754A0080A7C200DD
:082FD100E522640C6002D2014C
:102FD90002314B752C02A200B3400302308E741FDC
:102FE90090F000F07401123FD090F100E0540864B1
:102FF900006008741190F000F08006741090F000E1
:10300900F0754802122000742F90F000F07401123C
:103019003FD090F100E0540864006008742190F0FA
:1030290000F08006742090F000F07548021220002C
:10303900744F90F000F07401123FD090F100E05409
:103049000864006008744190F000F08006744090B4
:10305900F000F0754802122000748F90F000F074AF
:0E30690001123FD090F100E0540864006008AE
:0F307700748190F000F08006748090F000F07586
:103086004802122000022FDFC200E522640C600213
:10309600D20102314B752C03740290F400F07411C6
:1030A60090F300F0741190F302F074BC90F002F00B
:1030B6007548FA122000A200B3505F741190F30213
:1030C600F090F001E05420B4000A7480454A90F074
:1030D60000F0804490F302E4F0749290F003F074F0
:1030E60001123FD090F000E0540F903E39123FE0BD
:0A30F600E493F54A748290F003F0B1
:103100007401123FD074BC90F002F090F001E054D2
:103110002064006005A200B34002800280ED809C24
:10312000C200E522640C6002D201801F752C6390FE
:10313000F400E4F0743C90F002F0741090F202F0AD
:0B31400090F302E4F07548FA12200042
:0C320300022F6A022FDC02309B02312CEB
:04314B00022F5122DC
:103F0000748290F003F0749B90F103F0749290F23D
:103F100003F0748290F303F0748B90F403F0E52ABD
:103F2000903F49F8282873122018801C1220E8803E
:103F30001712235E8012122785800D1228DA80085E
:083F4000122B7F8003122F39C0
:103F4900023F27023F2C023F31023F36023F3B022C
:053F59003F40023F455E
:013F48002256
:093FE0002582F5825002058322BE
:083FF0000806B60002180622C3
:103FD000600D782B023FDA007830D8FED5E0F82269
:00414F016F
